:0200000480007A
:10000000970500009385C506130540006B10B500E9
:10001000EF00C005130510006B000500138581C3B8
:100020001386C1C33306A64093050000EF00901D60
:10003000171500001305858DEF00D008EF00D012D2
:10004000130540006B000500EF0010046F00D0089E
:10005000B707000093870700638807003715008003
:10006000130585906F00100667800000130540009F
:100070006B0005009711000093814179F32610026F
:100080009396A601732600029315A6001316260068
:1000900037F1FF6F3301B1403301D1403301C1006B
:1000A000F326100263860600130500006B000500AE
:1000B0006780000013052000D77285001305A0009B
:1000C00023A0A50023A0A50207E005125700000207
:1000D00027E0050267800000130101FD232681024D
:1000E00013040103232EA4FC232CB4FC232AC4FCF8
:1000F0008327C4FD83A707002326F4FE930744FD4E
:100100002322F4FE832744FE03C707008327C4FE8F
:100110002380E7008327C4FE93871700032744FE4C
:10012000034717002380E7008327C4FE9387270037
:10013000032744FE034727002380E7008327C4FEEC
:1001400093873700032744FE034737002380E700E7
:100150008327C4FE938747002326F4FE232404FE4E
:100160006F004003832784FE032784FDB307F70055
:1001700003C707008327C4FE2380E7008327C4FE4C
:10018000938717002326F4FE832784FE93871700A6
:100190002324F4FE832744FD032784FEE344F7FC75
:1001A0008327C4FE2320F4FE832704FE93F7370041
:1001B000032704FEB307F7002320F4FE832704FE81
:1001C0002326F4FE8327C4FD0327C4FE23A0E700F3
:1001D000130000000324C102130101036780000023
:1001E000130101FC232E8102130401042326A4FC25
:1001F0002324B4FC8327C4FC83A707002326F4FE32
:100200009307C4FD2322F4FE8327C4FE03C707001F
:10021000832744FE2380E700832744FE938717004B
:100220000327C4FE034717002380E700832744FE0B
:10023000938727000327C4FE034727002380E70096
:10024000832744FE938737000327C4FE0347370004
:100250002380E7008327C4FE938747002326F4FE0C
:10026000232404FE6F004003832784FE032784FCBD
:10027000B307F7000327C4FE034707002380E70006
:100280008327C4FE938717002326F4FE832784FE6A
:10029000938717002324F4FE8327C4FD032784FEDD
:1002A000E344F7FC8327C4FE2320F4FE832704FEE7
:1002B00093F73700032704FEB307F7002320F4FE6B
:1002C000832704FE2326F4FE8327C4FC0327C4FEF1
:1002D00023A0E700130000000324C103130101045D
:1002E00067800000130101FF232681001304010130
:1002F000130000000324C100130101016780000006
:10030000130101FE232E8100130401022326A4FE03
:100310002324B4FE832784FE3727000023A2E700AE
:1003200093070000138507000324C1011301010294
:1003300067800000130101FE232E1100232C810091
:10034000130401022326A4FEB7170080138507CDEE
:10035000EF00C04F93071000138507008320C101F1
:10036000032481011301010267800000130101FDD4
:10037000232611022324810213040103232EA4FC4B
:10038000232CB4FC232AC4FCB70700712326F4FEF7
:10039000B70700722324F4FE930730002322F4FEF3
:1003A000130744FE9307C4FE13064000930507009D
:1003B00013850700EFF05FD21307C4FD9307C4FE57
:1003C000130640009305070013850700EFF0DFD008
:1003D000130784FD9307C4FE13064000930507002E
:1003E00013850700EFF05FCF130744FD9307C4FEAA
:1003F000130640009305070013850700EFF0DFCDDB
:1004000083A7C1C2E7800700130704FE930784FE99
:100410009305070013850700EFF09FDC832704FE98
:10042000138507008320C102032481021301010305
:1004300067800000130101FD23261102232481029D
:1004400013040103232EA4FC232CB4FC232AC4FC94
:10045000B70700712324F4FEB70700722326F4FEC9
:10046000930740002322F4FE130744FE930784FE03
:10047000130640009305070013850700EFF0DFC562
:100480001307C4FD930784FE13064000930507007D
:1004900013850700EFF05FC4130784FD930784FE04
:1004A000130640009305070013850700EFF0DFC235
:1004B000130744FD930784FE1306400093050700CD
:1004C00013850700EFF05FC183A7C1C2E780070073
:1004D000832744FD138507008320C1020324810282
:1004E0001301010367800000130101FD232611029F
:1004F0002324810213040103232EA4FC232CB4FC27
:10050000232AC4FCB70700712326F4FE930750008A
:100510002324F4FE130784FE9307C4FE1306400051
:100520009305070013850700EFF01FBB1307C4FDF9
:100530009307C4FE130640009305070013850700C8
:10054000EFF09FB99307C4FE032644FD832584FD85
:1005500013850700EFF05FB883A7C1C2E7800700EB
:10056000832744FD138507008320C10203248102F1
:100570001301010367800000130101FD232681029E
:1005800013040103232EA4FC8327C4FD63D80700B2
:100590008327C4FDB307F040232EF4FC0327C4FDDA
:1005A000B73700009387078063D8E700B7370000AC
:1005B00093870780232EF4FC83A701C32326F4FE30
:1005C00003A701C38327C4FD3307F70023A8E1C2B3
:1005D0008327C4FE138507000324C102130101030E
:1005E00067800000130101FE232E1100232C8100DF
:1005F000130401022326A4FE13050000EF00001ED1
:10060000130000008320C1010324810113010102B2
:1006100067800000130101FD2326110223248102BB
:1006200013040103232EA4FC232CB4FC232AC4FCB2
:10063000B70700712326F4FEB70700722324F4FEE7
:10064000930770002322F4FE130744FE9307C4FEB1
:10065000130640009305070013850700EFF0DFA79E
:100660001307C4FD9307C4FE13064000930507005B
:1006700013850700EFF05FA6130784FD9307C4FE00
:10068000130640009305070013850700EFF0DFA471
:10069000130744FD9307C4FE1306400093050700AB
:1006A00013850700EFF05FA383A7C1C2E7800700AF
:1006B000130704FE930784FE9305070013850700C4
:1006C000EFF01FB2832704FE138507008320C102C9
:1006D000032481021301010367800000130101FF5D
:1006E000232611002324810013040101B717008081
:1006F000138547CEEF008015130000008320C10052
:10070000032481001301010167800000130101FF30
:10071000232611002324810013040101EF00800E21
:1007200093070500138507008320C100032481007F
:100730001301010167800000130101FF232611004E
:100740002324810013040101B7170080138587D08B
:10075000EF00C00F130000008320C10003248100BC
:100760001301010167800000130101FF232611001E
:100770002324810013040101B71700801385C7D219
:10078000EF00C00C83A781C39386170023ACD1C2AE
:10079000138507008320C100032481001301010198
:1007A00067800000130101FF23261100232481002C
:1007B00013040101B7170080138587D5EF000009E6
:1007C000130000008320C1000324810013010101F4
:1007D000678000006B10B500678000006B000500AB
:1007E000678000006B40B500678000006B2005004B
:1007F000678000006B3000006780000073251002E6
:100800006780000073250002678000001305400028
:100810006B000500F32610029396F6007326000283
:100820009315A6001316260037F1FF6F3301B14070
:100830003301D1403301C100F32610026386060064
:10084000130500006B00050067800000130141FFE5
:10085000232011002322B100834505006388050091
:10086000EF00C001130515006FF01FFF832001008A
:10087000832541001301C10067800000B702010019
:1008800023A0B20067800000130101FF232611009E
:10089000232481001304010113051000EFF01FF45D
:1008A000EFF05F8113050000EFF05FF3130000002D
:1008B000138507008320C100032481001301010177
:1008C00067800000930505009306000013060000F2
:1008D000130500006F00C020130101FF9305000005
:1008E000232481002326110013040500EF00C028F3
:1008F00003A581C28327C50363840700E78007003F
:1009000013050400EFF01FCE130101FF2324810023
:100910002322910037140080B7140080938744008D
:10092000130444003304F4402326110013542440DC
:1009300063020402931424009384C4FFB384F4007C
:1009400083A704001304F4FF9384C4FFE780070027
:10095000E31804FE8320C1000324810083244100A6
:100960001301010167800000130101FF23248100AE
:1009700023202101371400803719008093070400D9
:10098000130909003309F94023261100232291009D
:100990001359294063000902130404009304000062
:1009A000832704009384140013044400E7800700A5
:1009B000E31899FE3714008037190080930704006C
:1009C000130949003309F94013592940630009020A
:1009D000130404009304000083270400938414008C
:1009E00013044400E7800700E31899FE8320C10048
:1009F0000324810083244100032901001301010124
:100A0000678000001303F00013070500637EC30234
:100A10009377F7006390070A63920508937606FFC1
:100A20001376F600B386E6002320B7002322B70032
:100A30002324B7002326B70013070701E366D7FE78
:100A40006314060067800000B306C3409396260037
:100A500097020000B38656006780C6002307B700E0
:100A6000A306B7002306B700A305B7002305B70008
:100A7000A304B7002304B700A303B7002303B70000
:100A8000A302B7002302B700A301B7002301B700F8
:100A9000A300B7002300B7006780000093F5F50FAF
:100AA00093968500B3E5D50093960501B3E5D5008F
:100AB0006FF0DFF69396270097020000B38656008A
:100AC00093820000E78006FA93800200938707FF75
:100AD0003307F7403306F600E378C3F66FF0DFF331
:100AE00003A781C283278714638C070403A74700E9
:100AF0001308F001634EE806131827006306050289
:100B0000338307012324C30883A887181306100022
:100B10003316E600B3E8C80023A417192324D31022
:100B2000930620006304D5021307170023A2E700F1
:100B3000B387070123A4B7001305000067800000F6
:100B40009307C7142324F7146FF05FFA83A6C7181E
:100B50001307170023A2E70033E6C60023A6C71831
:100B6000B387070123A4B7001305000067800000C6
:100B70001305F0FF67800000130101FD23248101AC
:100B800003AC81C2232E3101232C4101232A5101C0
:100B900023286101232611022324810223229102AA
:100BA0002320210323267101930A0500138B0500DE
:100BB000130A10009309F0FF03298C14630809023B
:100BC000832449001384F4FF6342040293942400B5
:100BD000B304990063040B0483A744106380670582
:100BE0001304F4FF9384C4FFE31634FF8320C1028F
:100BF0000324810283244102032901028329C101C4
:100C0000032A8101832A4101032B0101832BC100A7
:100C1000032C810013010103678000008327490032
:100C200083A644009387F7FF638A870423A2040006
:100C3000E38806FA8327891833178A00832B490033
:100C4000B377F700639E0700E7800600832749001B
:100C5000E39477F783278C14E38427F96FF0DFF5AB
:100C60008327C91883A544083377F700631C07005E
:100C700013850A00E78006006FF05FFD23228900DC
:100C80006FF01FFB13850500E78006006FF01FFC67
:100C9000300000003100000032000000330000008E
:100CA000340000003500000036000000370000006E
:100CB0003800000039000000610000006200000000
:100CC0006300000064000000650000006600000092
:100CD00048656C6C6F2066726F6D205F697361741C
:100CE00074790A004552524F523A205F6B696C6C1E
:100CF000206E6F742079657420696D706C656D6508
:100D00006E7465640A0000004552524F523A205FEB
:100D1000756E6C696E6B206E6F74207965742069D6
:100D20006D706C656D656E7465640A004552524F56
:100D3000523A205F67657474696D656F66646179A6
:100D4000206E6F742079657420696D706C656D65B7
:100D50006E7465640A0000004552524F523A205F9B
:100D60006C696E6B206E6F742079657420696D708C
:0A0D70006C656D656E7465640A0021
:04100000500000801C
:1010080000000000F41200805C130080C41300800C
:1010180000000000000000000000000000000000C8
:1010280000000000000000000000000000000000B8
:1010380000000000000000000000000000000000A8
:101048000000000000000000000000000000000098
:101058000000000000000000000000000000000088
:101068000000000000000000000000000000000078
:101078000000000000000000000000000000000068
:101088000000000000000000000000000000000058
:101098000000000000000000000000000000000048
:1010A8000000000000000000010000000000000037
:1010B8000E33CDAB34126DE6ECDE05000B000000FC
:1010C8000000000000000000000000000000000018
:1010D8000000000000000000000000000000000008
:1010E80000000000000000000000000000000000F8
:1010F80000000000000000000000000000000000E8
:101430000810008000000070000000100000002074
:040000058000000077
:00000001FF
